******************************************************************************
                  TI ARM Linker PC v5.1.5                      
******************************************************************************
>> Linked Tue Mar 10 08:59:40 2015

OUTPUT FILE NAME:   <EDCU_TMS570LS1227.v0100.out>
ENTRY POINT SYMBOL: "_c_int00"  address: 000147a4


MEMORY CONFIGURATION

         name            origin    length      used     unused   attr    fill
----------------------  --------  ---------  --------  --------  ----  --------
  VECTORS               00000000   00000020  00000020  00000000     X
  FLASH0                00000020   0013ffe0  000164a8  00129b38  R  X
  STACKS                08000000   00001500  00000000  00001500  RW  
  RAM                   08001500   0002eb00  000010fc  0002da04  RW  


SEGMENT ALLOCATION MAP

run origin  load origin   length   init length attrs members
----------  ----------- ---------- ----------- ----- -------
00000000    00000000    000164c8   000164c8    r-x
  00000000    00000000    00000020   00000020    r-x .intvecs
  00000020    00000020    00015c28   00015c28    r-x .text
  00015c48    00015c48    000005f0   000005f0    r-- .const
  00016238    00016238    00000290   00000290    r-- .cinit
08001500    08001500    000010fc   00000000    rw-
  08001500    08001500    00000e0c   00000000    rw- .bss
  0800230c    0800230c    000002f0   00000000    rw- .data


SECTION ALLOCATION MAP

 output                                  attributes/
section   page    origin      length       input sections
--------  ----  ----------  ----------   ----------------
.intvecs   0    00000000    00000020     
                  00000000    00000020     sys_intvecs.obj (.intvecs)

.text      0    00000020    00015c28     
                  00000020    00002ccc     sys_selftest.obj (.text)
                  00002cec    00002394     etpwm.obj (.text)
                  00005080    000018a4     dlsw_logic.obj (.text)
                  00006924    000015a8     dlsw_motorc.obj (.text)
                  00007ecc    000011ec     spi.obj (.text)
                  000090b8    0000107c     dlsw_move.obj (.text)
                  0000a134    00000bf4     dlsw_curve.obj (.text)
                  0000ad28    00000b7c     dlsw_force.obj (.text)
                  0000b8a4    00000b2c     dlsw_diagnose.obj (.text)
                  0000c3d0    00000b28     system.obj (.text)
                  0000cef8    00000afc     adc.obj (.text)
                  0000d9f4    00000a54     sys_vim.obj (.text)
                  0000e448    00000960     dlsw_obstacle.obj (.text)
                  0000eda8    00000904     pinmux.obj (.text)
                  0000f6ac    000008f4     het.obj (.text)
                  0000ffa0    000008d0     ecap.obj (.text)
                  00010870    00000864     dlsw_io.obj (.text)
                  000110d4    00000858     drv_spi.obj (.text)
                  0001192c    00000804     spi.obj (.text:retain)
                  00012130    0000074c     sci.obj (.text)
                  0001287c    00000634     esm.obj (.text)
                  00012eb0    00000630     rti.obj (.text)
                  000134e0    000004a0     sys_main.obj (.text)
                  00013980    00000484     gio.obj (.text)
                  00013e04    000003c4     sys_core.obj (.text)
                  000141c8    00000300     sys_mpu.obj (.text)
                  000144c8    000002dc     sys_vim.obj (.text:retain)
                  000147a4    00000270     sys_startup.obj (.text:retain)
                  00014a14    0000022c     drv.obj (.text)
                  00014c40    000001ec     dlsw_timer.obj (.text)
                  00014e2c    000001b8     notification.obj (.text)
                  00014fe4    00000198     ecap.obj (.text:retain)
                  0001517c    00000158     esm.obj (.text:retain)
                  000152d4    00000114     sys_pmu.obj (.text)
                  000153e8    000000e8     dabort.obj (.text)
                  000154d0    000000c0     drv_public.obj (.text)
                  00015590    000000b4     pi.obj (.text)
                  00015644    000000a4     adc.obj (.text:retain)
                  000156e8    0000009c     rtsv7R4_T_be_v3D16_eabi.lib : memcpy_t2.obj (.text)
                  00015784    00000098     gio.obj (.text:retain)
                  0001581c    00000094     rti.obj (.text:retain)
                  000158b0    00000094     rtsv7R4_T_be_v3D16_eabi.lib : auto_init.obj (.text)
                  00015944    00000078                                 : memset_t2.obj (.text)
                  000159bc    00000060                                 : copy_decompress_rle.obj (.text)
                  00015a1c    00000058                                 : i_div32.obj (.text)
                  00015a74    00000054                                 : u_div32.obj (.text)
                  00015ac8    00000048                                 : cpy_tbl.obj (.text)
                  00015b10    00000044                                 : exit.obj (.text)
                  00015b54    0000003c                                 : fmaxf.obj (.text)
                  00015b90    0000003c                                 : fminf.obj (.text)
                  00015bcc    0000003c                                 : xfdtest.obj (.text)
                  00015c08    00000014                                 : _lock.obj (.text)
                  00015c1c    00000012                                 : copy_zero_init.obj (.text:decompress:ZI)
                  00015c2e    0000000e                                 : copy_decompress_none.obj (.text:decompress:none)
                  00015c3c    00000006                                 : copy_decompress_rle.obj (.text:decompress:rle24)
                  00015c42    00000002     --HOLE-- [fill = 0]
                  00015c44    00000004     sys_phantom.obj (.text:retain)

.const     0    00015c48    000005f0     
                  00015c48    000003a0     het.obj (.const:het1PROGRAM)
                  00015fe8    00000200     sys_vim.obj (.const:s_vim_init)
                  000161e8    00000030     adc.obj (.const)
                  00016218    00000020     het.obj (.const)

.cinit     0    00016238    00000290     
                  00016238    0000026b     (.cinit..data.load) [load image, compression = rle]
                  000164a3    00000001     --HOLE-- [fill = 0]
                  000164a4    0000000c     (__TI_handler_table)
                  000164b0    00000008     (.cinit..bss.load) [load image, compression = zero_init]
                  000164b8    00000010     (__TI_cinit_table)

.bss       0    08001500    00000e0c     UNINITIALIZED
                  08001500    000006f4     sys_main.obj (.bss:drl)
                  08001bf4    000001c8     sys_main.obj (.bss:stEcmp)
                  08001dbc    00000194     sys_main.obj (.bss:stMtr)
                  08001f50    00000118     sys_main.obj (.bss:stDrv)
                  08002068    000000f0     sys_main.obj (.bss:mtr)
                  08002158    00000078     spi.obj (.bss:g_spiPacket_t)
                  080021d0    00000054     sys_main.obj (.bss:crv)
                  08002224    00000050     drv_spi.obj (.bss:ucReceiveBufferArray)
                  08002274    00000030     drv_spi.obj (.bss:ucSendBufferArray)
                  080022a4    00000028     sci.obj (.bss:g_sciTransfer_t)
                  080022cc    00000024     sys_main.obj (.bss:stPID)
                  080022f0    00000012     (.common:gstSPICmdStatus)
                  08002302    00000004     (.common:dataconfig1_t)
                  08002306    00000002     --HOLE--
                  08002308    00000004     (.common:delayval$1)

.data      0    0800230c    000002f0     UNINITIALIZED
                  0800230c    00000200     drv_public.obj (.data:crc16_table)
                  0800250c    00000092     sys_main.obj (.data:tmr)
                  0800259e    00000029     drv_spi.obj (.data)
                  080025c7    00000001     --HOLE--
                  080025c8    0000001e     sys_main.obj (.data)
                  080025e6    00000002     --HOLE--
                  080025e8    00000008     rtsv7R4_T_be_v3D16_eabi.lib : _lock.obj (.data)
                  080025f0    00000008                                 : exit.obj (.data)
                  080025f8    00000004     dlsw_motorc.obj (.data)


LINKER GENERATED COPY TABLES

__TI_cinit_table @ 000164b8 records: 2, size/record: 8, table size: 16
	.data: load addr=00016238, load size=0000026b bytes, run addr=0800230c, run size=000002f0 bytes, compression=rle
	.bss: load addr=000164b0, load size=00000008 bytes, run addr=08001500, run size=00000e0c bytes, compression=zero_init


LINKER GENERATED HANDLER TABLE

__TI_handler_table @ 000164a4 records: 3, size/record: 4, table size: 12
	index: 0, handler: __TI_zero_init
	index: 1, handler: __TI_decompress_rle24
	index: 2, handler: __TI_decompress_none


GLOBAL SYMBOLS: SORTED ALPHABETICALLY BY Name 

address    name
--------   ----
0000b1c0   AverageClsRsstnc
0000b300   AverageOpnRsstnc
00015b11   C$$EXIT
0000adac   CalculateClsRsstnc
0000affc   CalculateOpnRsstnc
00007914   CalculatePWMComp
000076fc   ClearMtrPrtctCntr
00007784   ClearSpeedFeedback
0000ad28   CnfgrClsSlopRsstnc
0000af78   CnfgrOpnSlopRsstnc
0000a134   CnfgrSpeedCurve
00007884   CntrlAcrPi
00007804   CntrlAsrPi
0000567c   CntrlCentralClose
0000530c   CntrlCentralOpen
000057c8   CntrlCloseObstcl
0000944c   CntrlClsMove
00005090   CntrlEmrgncyOprtn
00006168   CntrlEmrgncyResetClose
0000c3a8   CntrlFailRecordStack
00006798   CntrlFlashOprtn
00006610   CntrlFullyClosedOprtn
000066a4   CntrlFullyOpenedOprtn
0000a090   CntrlInhibitMove
00005d04   CntrlInitialClose
000067bc   CntrlIsolateOprtn
000061f0   CntrlIsolateResetClose
00009ea4   CntrlKeepMove
00005fd0   CntrlLeaveOutFailClose
00005d84   CntrlLostSpeedClose
000072ac   CntrlMotorStartStop
00007268   CntrlMtrProtection
000053d4   CntrlOpenObstcl
000090b8   CntrlOpnMove
00015590   CntrlPID
00007c4c   CntrlPWMOutput
00006598   CntrlPosSensorFailStop
00009818   CntrlReopnReclsMove
000064b8   CntrlReopncls
0000a6b4   CntrlSpdCurve
0000a008   CntrlStopMove
00005e64   CntrlSwitchFailClose
000067a8   CntrlTimeoutOprtn
0000630c   CntrlZerospdResetClose
00014b48   Config8301
00006964   DRV_Motor_start
000069ac   DRV_Motor_stop
00006a50   DRV_setupPwms
0000c280   DiagBrakeSysFail
0000bdbc   DiagClsObstcDtcFail
0000bb4c   DiagDoorClsdSWFail
0000ba48   DiagDoorLckdSWFail
0000bf34   DiagIntrnlRelayFail
0000c0e0   DiagLckDeviceFail
0000bfe0   DiagLeaveOutFail
0000b8a4   DiagMtrCrcutOpnFail
0000be88   DiagOpnObstcDtcFail
0000c298   DiagPdpintFail
0000bd64   DiagPosSensorFail
0000bc50   DiagUnlock3sFail
00014dfc   DlyLogicTimer
00014a14   Drv_Init
00005744   DtctCloseOBstclMode
0000e4a0   DtctDoorPosition
00006768   DtctFailCodePriority
0000c3bc   DtctFailRecord
00006788   DtctHardwareVerNum
0000e7d8   DtctMotorBlocked
0000eaf8   DtctMoveObstacle
0000528c   DtctOpenAuth
0000e5e8   DtctPositionBlocked
0000521c   DtctSelfServiceMode
00006778   DtctSoftwareVerNum
000108f0   FilterInput
00010978   FilterInput00
00010a1c   FilterInput01
00010ac0   FilterInput02
00010b64   FilterInput04
00010c08   FilterInput13
00010cac   FilterInput14
00010d50   FilterInputGIO00
00010dec   FilterInputGIO01
00010e90   FilterInputGIO02
00010f34   FilterMtrOverTmprtr
00005080   GetCmd
00007b84   GetHallValue
00007238   HandleGPTmr2PrdInt
0000c2e0   IntegrateFailTag
0001321c   IsdwdKeySequenceCorrect
00006924   MtrCtrInit
00006d18   PWM_clearIntFlag
00006cfc   PWM_clearSocAFlag
00006e00   PWM_disableChopping
000071e0   PWM_disableCounterLoad
00006dc4   PWM_disableInt
00006de4   PWM_disableTripZones
00006d6c   PWM_enableSocAPulse
00006ee0   PWM_setActionQual_CntDown_CmpA_PwmA
00006f18   PWM_setActionQual_CntUp_CmpA_PwmA
00007100   PWM_setClkDiv
00007050   PWM_setCount
00007200   PWM_setCounterMode
00006e20   PWM_setDeadBandFallingEdgeDelay
00006ea8   PWM_setDeadBandOutputMode
00006e70   PWM_setDeadBandPolarity
00006e48   PWM_setDeadBandRisingEdgeDelay
00007138   PWM_setHighSpeedClkDiv
00006ff8   PWM_setLoadMode_CmpA
00006fc0   PWM_setLoadMode_CmpB
00007030   PWM_setPeriod
000071a8   PWM_setPeriodLoad
00007070   PWM_setPhase
000070c8   PWM_setPhaseDir
00007090   PWM_setRunMode
00006f88   PWM_setShadowMode_CmpA
00006f50   PWM_setShadowMode_CmpB
00006d34   PWM_setSocAPeriod
00006d8c   PWM_setSocAPulseSrc
00007170   PWM_setSyncMode
00006a00   PWM_write_CmpA
00010870   ReadInputSignal
00007690   ReadMotorOffsetIdc
0000798c   ResetSpeedTimer
UNDEFED    SHT$$INIT_ARRAY$$Base
UNDEFED    SHT$$INIT_ARRAY$$Limit
00011450   SPI_DataInit
0001143c   SPI_Process
0000b440   SetCurrentLimit
0000a0a0   SetMtrRotationTimer
0000b694   SetPIPrmtr
00014ab0   SetupDRV
000089b4   SpiRxStatus
00008928   SpiTxStatus
080025cc   StartFlag
00014c40   Update100msTimer
00014cc4   Update10msTimer
00014d48   Update1msTimer
00007a80   UpdateCurrent
00010fd8   UpdateInputSignal
00014db4   UpdateMtrRttnTimer
000079a8   UpdateSpeed
0000e51c   UpdateTotalDistance
0000e448   UpdateZeroPoint
00015bcd   _FDtest
000164b8   __TI_CINIT_Base
000164c8   __TI_CINIT_Limit
000164a4   __TI_Handler_Table_Base
000164b0   __TI_Handler_Table_Limit
000141c0   __TI_PINIT_Base
000141c4   __TI_PINIT_Limit
000158b1   __TI_auto_init
080025f0   __TI_cleanup_ptr
00015c2f   __TI_decompress_none
00015c3d   __TI_decompress_rle24
080025f4   __TI_dtors_ptr
00000000   __TI_static_base__
00015c1d   __TI_zero_init
00015a1c   __aeabi_idivmod
00015945   __aeabi_memclr
00015945   __aeabi_memclr4
00015945   __aeabi_memclr8
000156e9   __aeabi_memcpy
000156e9   __aeabi_memcpy4
000156e9   __aeabi_memcpy8
00015947   __aeabi_memset
00015947   __aeabi_memset4
00015947   __aeabi_memset8
00015a74   __aeabi_uidivmod
ffffffff   __binit__
ffffffff   __c_args__
000147a4   _c_int00
000140b8   _coreClearAuxiliaryDataFault_
000140d4   _coreClearAuxiliaryInstructionFault_
00014080   _coreClearDataFaultAddress_
00014048   _coreClearDataFault_
0001409c   _coreClearInstructionFaultAddress_
00014064   _coreClearInstructionFault_
00013fac   _coreDisableEventBusExport_
00014010   _coreDisableFlashEcc_
00013fdc   _coreDisableRamEcc_
00013f94   _coreEnableEventBusExport_
00013ff4   _coreEnableFlashEcc_
00014028   _coreEnableIrqVicOffset_
00013fc4   _coreEnableRamEcc_
00013f7c   _coreEnableVfp_
000140b0   _coreGetAuxiliaryDataFault_
000140cc   _coreGetAuxiliaryInstructionFault_
00014078   _coreGetDataFaultAddress_
00014040   _coreGetDataFault_
00014094   _coreGetInstructionFaultAddress_
0001405c   _coreGetInstructionFault_
00013e04   _coreInitRegisters_
00013f10   _coreInitStackPointer_
000153e8   _dabort
000140f0   _disable_FIQ_interrupt_
000140f8   _disable_IRQ_interrupt_
000140e8   _disable_interrupt_
00014100   _enable_interrupt_
00014190   _errata_CORTEXR4_57_
000141a8   _errata_CORTEXR4_66_
00014108   _esmCcmErrorsClear_
00013f5c   _getCPSRValue_
00013f64   _gotoCPUIdle_
080025e8   _lock
00014470   _mpuAreRegionsSeparate_
0001444c   _mpuDisableBackgroundRegion_
00014414   _mpuDisable_
00014434   _mpuEnableBackgroundRegion_
000143f4   _mpuEnable_
00014464   _mpuGetNumberOfRegions_
00014494   _mpuGetRegionBaseAddress_
000144b4   _mpuGetRegionPermission_
000144a8   _mpuGetRegionType_
00014484   _mpuGetRegion_
000141c8   _mpuInit_
0001448c   _mpuSetRegionBaseAddress_
000144c0   _mpuSetRegionSizeRegister_
0001449c   _mpuSetRegionTypeAndPermission_
0001447c   _mpuSetRegion_
00015c17   _nop
0001533c   _pmuDisableCountersGlobal_
00015324   _pmuEnableCountersGlobal_
000153bc   _pmuGetCycleCount_
000153c4   _pmuGetEventCount_
000153d4   _pmuGetOverflow_
000152d4   _pmuInit_
00015384   _pmuResetCounters_
00015354   _pmuResetCycleCounter_
0001536c   _pmuResetEventCounters_
000153ac   _pmuSetCountEvent_
0001539c   _pmuStartCounters_
000153a4   _pmuStopCounters_
00015c0f   _register_lock
00015c09   _register_unlock
080025ec   _unlock
00015b15   abort
0000d784   adc1GetConfigValue
00015644   adc1Group1Interrupt
00015690   adc1Group2Interrupt
0000124c   adc1ParityCheck
00001314   adc2ParityCheck
0000d358   adcCalibration
0000d724   adcDisableNotification
0000d6d4   adcEnableNotification
0000d128   adcGetData
0000d76c   adcGetEVTPin
0000cef8   adcInit
0000d328   adcIsConversionComplete
0000d2f8   adcIsFifoFull
0000d534   adcMidPointCalibration
000137a0   adcNotification
0000d100   adcResetFiFo
0000d74c   adcSetEVTPin
0000d054   adcStartConversion
0000d0d8   adcStopConversion
ffffffff   binit
000013f0   can1ParityCheck
000014c8   can2ParityCheck
00001590   can3ParityCheck
00014ea8   canErrorNotification
00014ed0   canMessageNotification
00014ebc   canStatusChangeNotification
0000fcb8   capGetSignal
080025ce   capIntTimes
00000030   ccmSelfCheck
000026ec   ccmr4GetConfigValue
00000918   checkB0RAMECC
00000b08   checkB1RAMECC
00001bf8   checkClockMonitor
00000cf8   checkFlashECC
00001cd4   checkFlashEEPROMECC
00001e6c   checkPLL1Slip
00001f6c   checkPLL2Slip
00002030   checkRAMAddrParity
000019b0   checkRAMECC
00002150   checkRAMUERRTest
0000079c   checkefcSelfTest
080025f8   clearSpdTimer
00015ac9   copy_in
080025c8   count_1ms
00000234   cpuSelfTest
00000ddc   cpuSelfTestFail
000154d0   crc16
00000dd4   custom_dabort
08002302   dataconfig1_t
00015548   delay
00002b48   disableParity
00014fd0   dmaGroupANotification
00000e8c   dmaParityCheck
080025d4   drvHandle
00013284   dwdClearFlag
000131b8   dwdCounterEnable
00013200   dwdGenerateSysReset
00013250   dwdGetStatus
00013294   dwdGetViolationStatus
0001313c   dwdInit
000131e4   dwdReset
000131c8   dwdSetPreload
000131ac   dwwdGetCurrentDownCounter
00013164   dwwdInit
00010498   ecap1GetConfigValue
00014fe4   ecap1Interrupt
0001052c   ecap2GetConfigValue
0001505c   ecap2Interrupt
000105c0   ecap3GetConfigValue
000150d4   ecap3nterrupt
00010654   ecap4GetConfigValue
000106e8   ecap5GetConfigValue
0001077c   ecap6GetConfigValue
00010418   ecapClearFlag
00010378   ecapDisableAPWMMode
00010268   ecapDisableCapture
00010060   ecapDisableCounterLoadOnSync
000103c4   ecapDisableInterrupt
0001030c   ecapEnableAPWMmode
00010248   ecapEnableCapture
00010030   ecapEnableCounterLoadOnSync
0001039c   ecapEnableInterrupt
00010438   ecapGetCAP1
00010450   ecapGetCAP2
00010468   ecapGetCAP3
00010480   ecapGetCAP4
000103f4   ecapGetEventStatus
0000ffa0   ecapInit
00013854   ecapNotification
000100c0   ecapSetCaptureEvent1
0001010c   ecapSetCaptureEvent2
0001015c   ecapSetCaptureEvent3
000101ac   ecapSetCaptureEvent4
000101fc   ecapSetCaptureMode
00010010   ecapSetCounter
00010084   ecapSetEventPrescaler
000102d0   ecapSetSyncOut
0001028c   ecapStartCounter
000102ac   ecapStopCounter
080025d8   ecmpHandle
0000fc78   edgeDisableNotification
0000fc3c   edgeEnableNotification
0000fc10   edgeGetCounter
00014f70   edgeNotification
0000fbe4   edgeResetCounter
00000640   efcCheck
00002654   efcGetConfigValue
00000774   efcSelfTest
000006c8   efcStuckZeroTest
00002ac0   enableParity
0000275c   errata_PBIST_4
00012a2c   esmActivateNormalOperation
00012b18   esmClearStatus
00012b58   esmClearStatusBuffer
000129f0   esmDisableError
00012a68   esmDisableInterrupt
000129c4   esmEnableError
00012a3c   esmEnableInterrupt
00012c78   esmEnterSelfTest
000129a8   esmError
00012d50   esmGetConfigValue
00012ba4   esmGetStatus
00012c18   esmGetStatusBuffer
00014e2c   esmGroup1Notification
00014e3c   esmGroup2Notification
0001517c   esmHighInterrupt
0001287c   esmInit
00012d00   esmSelfTestStatus
00012b84   esmSetCounterPreloadValue
00012a94   esmSetInterruptLevel
00012a1c   esmTriggerErrorPinReset
00003960   etpwm1GetConfigValue
00003ce8   etpwm2GetConfigValue
00003fdc   etpwm3GetConfigValue
000042bc   etpwm4GetConfigValue
0000459c   etpwm5GetConfigValue
00004884   etpwm6GetConfigValue
00004b94   etpwm7GetConfigValue
00003894   etpwmClearEventFlag
00003664   etpwmClearTripCondition
00003684   etpwmClearTripInterruptFlag
00003528   etpwmDisableChopping
000032f4   etpwmDisableCmpAShadowMode
00003354   etpwmDisableCmpBShadowMode
00003184   etpwmDisableCounterLoadOnSync
000034a8   etpwmDisableDeadband
00003858   etpwmDisableInterrupt
00003734   etpwmDisableSOCA
000037cc   etpwmDisableSOCB
000030f0   etpwmDisableTimebasePeriodShadowMode
00003634   etpwmDisableTripInterrupt
0000356c   etpwmDisableTripZoneSources
000034f4   etpwmEnableChopping
000032b8   etpwmEnableCmpAShadowMode
00003314   etpwmEnableCmpBShadowMode
00003134   etpwmEnableCounterLoadOnSync
00003454   etpwmEnableDeadBand
000038d4   etpwmEnableDigitalCompareEvents
000037ec   etpwmEnableInterrupt
000036c0   etpwmEnableSOCA
00003758   etpwmEnableSOCB
00003110   etpwmEnableTimebasePeriodShadowMode
0000360c   etpwmEnableTripInterrupt
00003544   etpwmEnableTripZoneSources
000036a0   etpwmForceTripEvent
0000387c   etpwmGetEventStatus
00002cec   etpwmInit
00014f98   etpwmNotification
00003374   etpwmSetActionQualPwmA
000033e4   etpwmSetActionQualPwmB
00003068   etpwmSetClkDiv
00003278   etpwmSetCmpA
00003298   etpwmSetCmpB
000030d0   etpwmSetCount
000031e4   etpwmSetCounterMode
000034c4   etpwmSetDeadBandDelay
00003240   etpwmSetRunMode
000031a8   etpwmSetSyncOut
000030b0   etpwmSetTimebasePeriod
0000359c   etpwmSetTripAction
00002fd4   etpwmStartTBCLK
00003020   etpwmStopTBCLK
000038b4   etpwmTriggerEvent
00003220   etpwmTriggerSWSync
00014fa8   etpwmTripNotification
00015b1d   exit
00015b55   fmaxf
000022b4   fmcBus1ParityCheck
0000083c   fmcBus2Check
00000878   fmcECCcheck
00015b91   fminf
00013be0   gioDisableNotification
00013b78   gioEnableNotification
00013ae0   gioGetBit
00013c48   gioGetConfigValue
00013b08   gioGetPort
00015784   gioHighLevelInterrupt
00013980   gioInit
00014ee4   gioNotification
00013a70   gioSetBit
00013a50   gioSetDirection
00013ac0   gioSetPort
00013b20   gioToggleBit
080022f0   gstSPICmdStatus
080025be   gucCmdFrameType
080025c1   gucSendDataOK
080025c2   gucSpiArmToDspSpiFault
080025bf   gucSpiRevCmpltFlag
080025c0   gucSpiRevOKFlag
0000fdc4   het1GetConfigValue
00000f38   het1ParityCheck
000010a0   het2ParityCheck
0000fdac   hetGetTimestamp
0000f6ac   hetInit
00014f84   hetNotification
0000fd90   hetResetTimestamp
00000fe4   htu1ParityCheck
0000119c   htu2ParityCheck
00014ef8   i2cNotification
00014f0c   linNotification
000134e0   main
0000c50c   mapClocks
000156e9   memcpy
00000174   memoryInit
00014e4c   memoryPort0TestFailNotification
00014e68   memoryPort1TestFailNotification
0001594d   memset
0001192c   mibspi1HighLevelInterrupt
00001664   mibspi1ParityCheck
0000176c   mibspi3ParityCheck
00011dfc   mibspi5LowLevelInterrupt
00001890   mibspi5ParityCheck
080025d0   mtrHandle
0000eda8   muxInit
000023e0   pbistFail
00002460   pbistGetConfigValue
000005a8   pbistIsTestCompleted
000005c4   pbistIsTestPassed
000005f8   pbistPortTestStatus
000004ac   pbistRun
000002cc   pbistSelfCheck
00000578   pbistStop
0000c4b8   periphInit
00015c44   phantomInterrupt
080025dc   piHandle
0000f28c   pinmuxGetConfigValue
0000fbb4   pwmDisableNotification
0000fb6c   pwmEnableNotification
0000fa8c   pwmGetSignal
00014f58   pwmNotification
0000f7d4   pwmSetDuty
0000f910   pwmSetSignal
0000f76c   pwmStart
0000f7a0   pwmStop
00000000   resetEntry
0001581c   rtiCompare2Interrupt
00015864   rtiCompare3Interrupt
00013344   rtiDisableNotification
0001331c   rtiEnableNotification
00013360   rtiGetConfigValue
000130b0   rtiGetCurrentTick
00013088   rtiGetPeriod
00012eb0   rtiInit
000138ec   rtiNotification
00012ffc   rtiResetCounter
00013060   rtiSetPeriod
00012fa4   rtiStartCounter
00012fd0   rtiStopCounter
000125dc   sciDisableLoopback
00012668   sciDisableNotification
000125a8   sciEnableLoopback
00012600   sciEnableNotification
000126d0   sciGetConfigValue
00012130   sciInit
00012458   sciIsIdleDetected
0001243c   sciIsRxReady
000122bc   sciIsTxReady
00014f20   sciNotification
000124d0   sciReceive
000124a4   sciReceiveByte
00012474   sciRxError
00012308   sciSend
000122d8   sciSendByte
0001223c   sciSetBaudrate
0001221c   sciSetFunctional
00000020   selftestFailNotification
0000c478   setupFlash
0000c3d0   setupPLL
00008aec   spi1GetConfigValue
00008c7c   spi4GetConfigValue
00011b94   spi4HighLevelInterrupt
00008e58   spi5GetConfigValue
00008a74   spiDisableLoopback
00008ac0   spiDisableNotification
00008a40   spiEnableLoopback
00008a90   spiEnableNotification
0001150c   spiEndNotification
00008390   spiGetData
00007ecc   spiInit
00014f34   spiNotification
00008274   spiReceiveData
000087e8   spiSendAndGetData
000085b4   spiSendData
00008254   spiSetFunctional
000086ac   spiTransmitAndReceiveData
00008488   spiTransmitData
0000ccf0   sramGetConfigValue
08001f50   stDrv
08001bf4   stEcmp
08001dbc   stMtr
080022cc   stPID
000025ac   stcGetConfigValue
000001b8   stcSelfCheck
00000dd8   stcSelfCheckFail
0000c730   systemGetConfigValue
0000c634   systemInit
0000c700   systemPowerDown
0000cb44   tcmflashGetConfigValue
0000c430   trimLPO
080025ae   ucRXbuffer
08002224   ucReceiveBufferArray
08002274   ucSendBufferArray
0800259e   ucTXbuffer
0000dac8   vimChannelMap
0000dd2c   vimDisableInterrupt
0000db64   vimEnableInterrupt
0000ddd8   vimGetConfigValue
0000d9f4   vimInit
00000de0   vimParityCheck
000144c8   vimParityErrorHandler


GLOBAL SYMBOLS: SORTED BY Symbol Address 

address    name
--------   ----
00000000   __TI_static_base__
00000000   resetEntry
00000020   selftestFailNotification
00000030   ccmSelfCheck
00000174   memoryInit
000001b8   stcSelfCheck
00000234   cpuSelfTest
000002cc   pbistSelfCheck
000004ac   pbistRun
00000578   pbistStop
000005a8   pbistIsTestCompleted
000005c4   pbistIsTestPassed
000005f8   pbistPortTestStatus
00000640   efcCheck
000006c8   efcStuckZeroTest
00000774   efcSelfTest
0000079c   checkefcSelfTest
0000083c   fmcBus2Check
00000878   fmcECCcheck
00000918   checkB0RAMECC
00000b08   checkB1RAMECC
00000cf8   checkFlashECC
00000dd4   custom_dabort
00000dd8   stcSelfCheckFail
00000ddc   cpuSelfTestFail
00000de0   vimParityCheck
00000e8c   dmaParityCheck
00000f38   het1ParityCheck
00000fe4   htu1ParityCheck
000010a0   het2ParityCheck
0000119c   htu2ParityCheck
0000124c   adc1ParityCheck
00001314   adc2ParityCheck
000013f0   can1ParityCheck
000014c8   can2ParityCheck
00001590   can3ParityCheck
00001664   mibspi1ParityCheck
0000176c   mibspi3ParityCheck
00001890   mibspi5ParityCheck
000019b0   checkRAMECC
00001bf8   checkClockMonitor
00001cd4   checkFlashEEPROMECC
00001e6c   checkPLL1Slip
00001f6c   checkPLL2Slip
00002030   checkRAMAddrParity
00002150   checkRAMUERRTest
000022b4   fmcBus1ParityCheck
000023e0   pbistFail
00002460   pbistGetConfigValue
000025ac   stcGetConfigValue
00002654   efcGetConfigValue
000026ec   ccmr4GetConfigValue
0000275c   errata_PBIST_4
00002ac0   enableParity
00002b48   disableParity
00002cec   etpwmInit
00002fd4   etpwmStartTBCLK
00003020   etpwmStopTBCLK
00003068   etpwmSetClkDiv
000030b0   etpwmSetTimebasePeriod
000030d0   etpwmSetCount
000030f0   etpwmDisableTimebasePeriodShadowMode
00003110   etpwmEnableTimebasePeriodShadowMode
00003134   etpwmEnableCounterLoadOnSync
00003184   etpwmDisableCounterLoadOnSync
000031a8   etpwmSetSyncOut
000031e4   etpwmSetCounterMode
00003220   etpwmTriggerSWSync
00003240   etpwmSetRunMode
00003278   etpwmSetCmpA
00003298   etpwmSetCmpB
000032b8   etpwmEnableCmpAShadowMode
000032f4   etpwmDisableCmpAShadowMode
00003314   etpwmEnableCmpBShadowMode
00003354   etpwmDisableCmpBShadowMode
00003374   etpwmSetActionQualPwmA
000033e4   etpwmSetActionQualPwmB
00003454   etpwmEnableDeadBand
000034a8   etpwmDisableDeadband
000034c4   etpwmSetDeadBandDelay
000034f4   etpwmEnableChopping
00003528   etpwmDisableChopping
00003544   etpwmEnableTripZoneSources
0000356c   etpwmDisableTripZoneSources
0000359c   etpwmSetTripAction
0000360c   etpwmEnableTripInterrupt
00003634   etpwmDisableTripInterrupt
00003664   etpwmClearTripCondition
00003684   etpwmClearTripInterruptFlag
000036a0   etpwmForceTripEvent
000036c0   etpwmEnableSOCA
00003734   etpwmDisableSOCA
00003758   etpwmEnableSOCB
000037cc   etpwmDisableSOCB
000037ec   etpwmEnableInterrupt
00003858   etpwmDisableInterrupt
0000387c   etpwmGetEventStatus
00003894   etpwmClearEventFlag
000038b4   etpwmTriggerEvent
000038d4   etpwmEnableDigitalCompareEvents
00003960   etpwm1GetConfigValue
00003ce8   etpwm2GetConfigValue
00003fdc   etpwm3GetConfigValue
000042bc   etpwm4GetConfigValue
0000459c   etpwm5GetConfigValue
00004884   etpwm6GetConfigValue
00004b94   etpwm7GetConfigValue
00005080   GetCmd
00005090   CntrlEmrgncyOprtn
0000521c   DtctSelfServiceMode
0000528c   DtctOpenAuth
0000530c   CntrlCentralOpen
000053d4   CntrlOpenObstcl
0000567c   CntrlCentralClose
00005744   DtctCloseOBstclMode
000057c8   CntrlCloseObstcl
00005d04   CntrlInitialClose
00005d84   CntrlLostSpeedClose
00005e64   CntrlSwitchFailClose
00005fd0   CntrlLeaveOutFailClose
00006168   CntrlEmrgncyResetClose
000061f0   CntrlIsolateResetClose
0000630c   CntrlZerospdResetClose
000064b8   CntrlReopncls
00006598   CntrlPosSensorFailStop
00006610   CntrlFullyClosedOprtn
000066a4   CntrlFullyOpenedOprtn
00006768   DtctFailCodePriority
00006778   DtctSoftwareVerNum
00006788   DtctHardwareVerNum
00006798   CntrlFlashOprtn
000067a8   CntrlTimeoutOprtn
000067bc   CntrlIsolateOprtn
00006924   MtrCtrInit
00006964   DRV_Motor_start
000069ac   DRV_Motor_stop
00006a00   PWM_write_CmpA
00006a50   DRV_setupPwms
00006cfc   PWM_clearSocAFlag
00006d18   PWM_clearIntFlag
00006d34   PWM_setSocAPeriod
00006d6c   PWM_enableSocAPulse
00006d8c   PWM_setSocAPulseSrc
00006dc4   PWM_disableInt
00006de4   PWM_disableTripZones
00006e00   PWM_disableChopping
00006e20   PWM_setDeadBandFallingEdgeDelay
00006e48   PWM_setDeadBandRisingEdgeDelay
00006e70   PWM_setDeadBandPolarity
00006ea8   PWM_setDeadBandOutputMode
00006ee0   PWM_setActionQual_CntDown_CmpA_PwmA
00006f18   PWM_setActionQual_CntUp_CmpA_PwmA
00006f50   PWM_setShadowMode_CmpB
00006f88   PWM_setShadowMode_CmpA
00006fc0   PWM_setLoadMode_CmpB
00006ff8   PWM_setLoadMode_CmpA
00007030   PWM_setPeriod
00007050   PWM_setCount
00007070   PWM_setPhase
00007090   PWM_setRunMode
000070c8   PWM_setPhaseDir
00007100   PWM_setClkDiv
00007138   PWM_setHighSpeedClkDiv
00007170   PWM_setSyncMode
000071a8   PWM_setPeriodLoad
000071e0   PWM_disableCounterLoad
00007200   PWM_setCounterMode
00007238   HandleGPTmr2PrdInt
00007268   CntrlMtrProtection
000072ac   CntrlMotorStartStop
00007690   ReadMotorOffsetIdc
000076fc   ClearMtrPrtctCntr
00007784   ClearSpeedFeedback
00007804   CntrlAsrPi
00007884   CntrlAcrPi
00007914   CalculatePWMComp
0000798c   ResetSpeedTimer
000079a8   UpdateSpeed
00007a80   UpdateCurrent
00007b84   GetHallValue
00007c4c   CntrlPWMOutput
00007ecc   spiInit
00008254   spiSetFunctional
00008274   spiReceiveData
00008390   spiGetData
00008488   spiTransmitData
000085b4   spiSendData
000086ac   spiTransmitAndReceiveData
000087e8   spiSendAndGetData
00008928   SpiTxStatus
000089b4   SpiRxStatus
00008a40   spiEnableLoopback
00008a74   spiDisableLoopback
00008a90   spiEnableNotification
00008ac0   spiDisableNotification
00008aec   spi1GetConfigValue
00008c7c   spi4GetConfigValue
00008e58   spi5GetConfigValue
000090b8   CntrlOpnMove
0000944c   CntrlClsMove
00009818   CntrlReopnReclsMove
00009ea4   CntrlKeepMove
0000a008   CntrlStopMove
0000a090   CntrlInhibitMove
0000a0a0   SetMtrRotationTimer
0000a134   CnfgrSpeedCurve
0000a6b4   CntrlSpdCurve
0000ad28   CnfgrClsSlopRsstnc
0000adac   CalculateClsRsstnc
0000af78   CnfgrOpnSlopRsstnc
0000affc   CalculateOpnRsstnc
0000b1c0   AverageClsRsstnc
0000b300   AverageOpnRsstnc
0000b440   SetCurrentLimit
0000b694   SetPIPrmtr
0000b8a4   DiagMtrCrcutOpnFail
0000ba48   DiagDoorLckdSWFail
0000bb4c   DiagDoorClsdSWFail
0000bc50   DiagUnlock3sFail
0000bd64   DiagPosSensorFail
0000bdbc   DiagClsObstcDtcFail
0000be88   DiagOpnObstcDtcFail
0000bf34   DiagIntrnlRelayFail
0000bfe0   DiagLeaveOutFail
0000c0e0   DiagLckDeviceFail
0000c280   DiagBrakeSysFail
0000c298   DiagPdpintFail
0000c2e0   IntegrateFailTag
0000c3a8   CntrlFailRecordStack
0000c3bc   DtctFailRecord
0000c3d0   setupPLL
0000c430   trimLPO
0000c478   setupFlash
0000c4b8   periphInit
0000c50c   mapClocks
0000c634   systemInit
0000c700   systemPowerDown
0000c730   systemGetConfigValue
0000cb44   tcmflashGetConfigValue
0000ccf0   sramGetConfigValue
0000cef8   adcInit
0000d054   adcStartConversion
0000d0d8   adcStopConversion
0000d100   adcResetFiFo
0000d128   adcGetData
0000d2f8   adcIsFifoFull
0000d328   adcIsConversionComplete
0000d358   adcCalibration
0000d534   adcMidPointCalibration
0000d6d4   adcEnableNotification
0000d724   adcDisableNotification
0000d74c   adcSetEVTPin
0000d76c   adcGetEVTPin
0000d784   adc1GetConfigValue
0000d9f4   vimInit
0000dac8   vimChannelMap
0000db64   vimEnableInterrupt
0000dd2c   vimDisableInterrupt
0000ddd8   vimGetConfigValue
0000e448   UpdateZeroPoint
0000e4a0   DtctDoorPosition
0000e51c   UpdateTotalDistance
0000e5e8   DtctPositionBlocked
0000e7d8   DtctMotorBlocked
0000eaf8   DtctMoveObstacle
0000eda8   muxInit
0000f28c   pinmuxGetConfigValue
0000f6ac   hetInit
0000f76c   pwmStart
0000f7a0   pwmStop
0000f7d4   pwmSetDuty
0000f910   pwmSetSignal
0000fa8c   pwmGetSignal
0000fb6c   pwmEnableNotification
0000fbb4   pwmDisableNotification
0000fbe4   edgeResetCounter
0000fc10   edgeGetCounter
0000fc3c   edgeEnableNotification
0000fc78   edgeDisableNotification
0000fcb8   capGetSignal
0000fd90   hetResetTimestamp
0000fdac   hetGetTimestamp
0000fdc4   het1GetConfigValue
0000ffa0   ecapInit
00010010   ecapSetCounter
00010030   ecapEnableCounterLoadOnSync
00010060   ecapDisableCounterLoadOnSync
00010084   ecapSetEventPrescaler
000100c0   ecapSetCaptureEvent1
0001010c   ecapSetCaptureEvent2
0001015c   ecapSetCaptureEvent3
000101ac   ecapSetCaptureEvent4
000101fc   ecapSetCaptureMode
00010248   ecapEnableCapture
00010268   ecapDisableCapture
0001028c   ecapStartCounter
000102ac   ecapStopCounter
000102d0   ecapSetSyncOut
0001030c   ecapEnableAPWMmode
00010378   ecapDisableAPWMMode
0001039c   ecapEnableInterrupt
000103c4   ecapDisableInterrupt
000103f4   ecapGetEventStatus
00010418   ecapClearFlag
00010438   ecapGetCAP1
00010450   ecapGetCAP2
00010468   ecapGetCAP3
00010480   ecapGetCAP4
00010498   ecap1GetConfigValue
0001052c   ecap2GetConfigValue
000105c0   ecap3GetConfigValue
00010654   ecap4GetConfigValue
000106e8   ecap5GetConfigValue
0001077c   ecap6GetConfigValue
00010870   ReadInputSignal
000108f0   FilterInput
00010978   FilterInput00
00010a1c   FilterInput01
00010ac0   FilterInput02
00010b64   FilterInput04
00010c08   FilterInput13
00010cac   FilterInput14
00010d50   FilterInputGIO00
00010dec   FilterInputGIO01
00010e90   FilterInputGIO02
00010f34   FilterMtrOverTmprtr
00010fd8   UpdateInputSignal
0001143c   SPI_Process
00011450   SPI_DataInit
0001150c   spiEndNotification
0001192c   mibspi1HighLevelInterrupt
00011b94   spi4HighLevelInterrupt
00011dfc   mibspi5LowLevelInterrupt
00012130   sciInit
0001221c   sciSetFunctional
0001223c   sciSetBaudrate
000122bc   sciIsTxReady
000122d8   sciSendByte
00012308   sciSend
0001243c   sciIsRxReady
00012458   sciIsIdleDetected
00012474   sciRxError
000124a4   sciReceiveByte
000124d0   sciReceive
000125a8   sciEnableLoopback
000125dc   sciDisableLoopback
00012600   sciEnableNotification
00012668   sciDisableNotification
000126d0   sciGetConfigValue
0001287c   esmInit
000129a8   esmError
000129c4   esmEnableError
000129f0   esmDisableError
00012a1c   esmTriggerErrorPinReset
00012a2c   esmActivateNormalOperation
00012a3c   esmEnableInterrupt
00012a68   esmDisableInterrupt
00012a94   esmSetInterruptLevel
00012b18   esmClearStatus
00012b58   esmClearStatusBuffer
00012b84   esmSetCounterPreloadValue
00012ba4   esmGetStatus
00012c18   esmGetStatusBuffer
00012c78   esmEnterSelfTest
00012d00   esmSelfTestStatus
00012d50   esmGetConfigValue
00012eb0   rtiInit
00012fa4   rtiStartCounter
00012fd0   rtiStopCounter
00012ffc   rtiResetCounter
00013060   rtiSetPeriod
00013088   rtiGetPeriod
000130b0   rtiGetCurrentTick
0001313c   dwdInit
00013164   dwwdInit
000131ac   dwwdGetCurrentDownCounter
000131b8   dwdCounterEnable
000131c8   dwdSetPreload
000131e4   dwdReset
00013200   dwdGenerateSysReset
0001321c   IsdwdKeySequenceCorrect
00013250   dwdGetStatus
00013284   dwdClearFlag
00013294   dwdGetViolationStatus
0001331c   rtiEnableNotification
00013344   rtiDisableNotification
00013360   rtiGetConfigValue
000134e0   main
000137a0   adcNotification
00013854   ecapNotification
000138ec   rtiNotification
00013980   gioInit
00013a50   gioSetDirection
00013a70   gioSetBit
00013ac0   gioSetPort
00013ae0   gioGetBit
00013b08   gioGetPort
00013b20   gioToggleBit
00013b78   gioEnableNotification
00013be0   gioDisableNotification
00013c48   gioGetConfigValue
00013e04   _coreInitRegisters_
00013f10   _coreInitStackPointer_
00013f5c   _getCPSRValue_
00013f64   _gotoCPUIdle_
00013f7c   _coreEnableVfp_
00013f94   _coreEnableEventBusExport_
00013fac   _coreDisableEventBusExport_
00013fc4   _coreEnableRamEcc_
00013fdc   _coreDisableRamEcc_
00013ff4   _coreEnableFlashEcc_
00014010   _coreDisableFlashEcc_
00014028   _coreEnableIrqVicOffset_
00014040   _coreGetDataFault_
00014048   _coreClearDataFault_
0001405c   _coreGetInstructionFault_
00014064   _coreClearInstructionFault_
00014078   _coreGetDataFaultAddress_
00014080   _coreClearDataFaultAddress_
00014094   _coreGetInstructionFaultAddress_
0001409c   _coreClearInstructionFaultAddress_
000140b0   _coreGetAuxiliaryDataFault_
000140b8   _coreClearAuxiliaryDataFault_
000140cc   _coreGetAuxiliaryInstructionFault_
000140d4   _coreClearAuxiliaryInstructionFault_
000140e8   _disable_interrupt_
000140f0   _disable_FIQ_interrupt_
000140f8   _disable_IRQ_interrupt_
00014100   _enable_interrupt_
00014108   _esmCcmErrorsClear_
00014190   _errata_CORTEXR4_57_
000141a8   _errata_CORTEXR4_66_
000141c0   __TI_PINIT_Base
000141c4   __TI_PINIT_Limit
000141c8   _mpuInit_
000143f4   _mpuEnable_
00014414   _mpuDisable_
00014434   _mpuEnableBackgroundRegion_
0001444c   _mpuDisableBackgroundRegion_
00014464   _mpuGetNumberOfRegions_
00014470   _mpuAreRegionsSeparate_
0001447c   _mpuSetRegion_
00014484   _mpuGetRegion_
0001448c   _mpuSetRegionBaseAddress_
00014494   _mpuGetRegionBaseAddress_
0001449c   _mpuSetRegionTypeAndPermission_
000144a8   _mpuGetRegionType_
000144b4   _mpuGetRegionPermission_
000144c0   _mpuSetRegionSizeRegister_
000144c8   vimParityErrorHandler
000147a4   _c_int00
00014a14   Drv_Init
00014ab0   SetupDRV
00014b48   Config8301
00014c40   Update100msTimer
00014cc4   Update10msTimer
00014d48   Update1msTimer
00014db4   UpdateMtrRttnTimer
00014dfc   DlyLogicTimer
00014e2c   esmGroup1Notification
00014e3c   esmGroup2Notification
00014e4c   memoryPort0TestFailNotification
00014e68   memoryPort1TestFailNotification
00014ea8   canErrorNotification
00014ebc   canStatusChangeNotification
00014ed0   canMessageNotification
00014ee4   gioNotification
00014ef8   i2cNotification
00014f0c   linNotification
00014f20   sciNotification
00014f34   spiNotification
00014f58   pwmNotification
00014f70   edgeNotification
00014f84   hetNotification
00014f98   etpwmNotification
00014fa8   etpwmTripNotification
00014fd0   dmaGroupANotification
00014fe4   ecap1Interrupt
0001505c   ecap2Interrupt
000150d4   ecap3nterrupt
0001517c   esmHighInterrupt
000152d4   _pmuInit_
00015324   _pmuEnableCountersGlobal_
0001533c   _pmuDisableCountersGlobal_
00015354   _pmuResetCycleCounter_
0001536c   _pmuResetEventCounters_
00015384   _pmuResetCounters_
0001539c   _pmuStartCounters_
000153a4   _pmuStopCounters_
000153ac   _pmuSetCountEvent_
000153bc   _pmuGetCycleCount_
000153c4   _pmuGetEventCount_
000153d4   _pmuGetOverflow_
000153e8   _dabort
000154d0   crc16
00015548   delay
00015590   CntrlPID
00015644   adc1Group1Interrupt
00015690   adc1Group2Interrupt
000156e9   __aeabi_memcpy
000156e9   __aeabi_memcpy4
000156e9   __aeabi_memcpy8
000156e9   memcpy
00015784   gioHighLevelInterrupt
0001581c   rtiCompare2Interrupt
00015864   rtiCompare3Interrupt
000158b1   __TI_auto_init
00015945   __aeabi_memclr
00015945   __aeabi_memclr4
00015945   __aeabi_memclr8
00015947   __aeabi_memset
00015947   __aeabi_memset4
00015947   __aeabi_memset8
0001594d   memset
00015a1c   __aeabi_idivmod
00015a74   __aeabi_uidivmod
00015ac9   copy_in
00015b11   C$$EXIT
00015b15   abort
00015b1d   exit
00015b55   fmaxf
00015b91   fminf
00015bcd   _FDtest
00015c09   _register_unlock
00015c0f   _register_lock
00015c17   _nop
00015c1d   __TI_zero_init
00015c2f   __TI_decompress_none
00015c3d   __TI_decompress_rle24
00015c44   phantomInterrupt
000164a4   __TI_Handler_Table_Base
000164b0   __TI_Handler_Table_Limit
000164b8   __TI_CINIT_Base
000164c8   __TI_CINIT_Limit
08001bf4   stEcmp
08001dbc   stMtr
08001f50   stDrv
08002224   ucReceiveBufferArray
08002274   ucSendBufferArray
080022cc   stPID
080022f0   gstSPICmdStatus
08002302   dataconfig1_t
0800259e   ucTXbuffer
080025ae   ucRXbuffer
080025be   gucCmdFrameType
080025bf   gucSpiRevCmpltFlag
080025c0   gucSpiRevOKFlag
080025c1   gucSendDataOK
080025c2   gucSpiArmToDspSpiFault
080025c8   count_1ms
080025cc   StartFlag
080025ce   capIntTimes
080025d0   mtrHandle
080025d4   drvHandle
080025d8   ecmpHandle
080025dc   piHandle
080025e8   _lock
080025ec   _unlock
080025f0   __TI_cleanup_ptr
080025f4   __TI_dtors_ptr
080025f8   clearSpdTimer
ffffffff   __binit__
ffffffff   __c_args__
ffffffff   binit
UNDEFED    SHT$$INIT_ARRAY$$Base
UNDEFED    SHT$$INIT_ARRAY$$Limit

[566 symbols]
